:020000040800F2
:10000000700B0024AD0200081518000893160008B4
:10001000B9020008C1030008E12000080000000048
:100020000000000000000000000000001918000897
:100030004D0400080000000017180008C918000847
:10004000C7020008C7020008C7020008C70200086C
:10005000C7020008C7020008C7020008C70200085C
:10006000C7020008C7020008C7020008C70200084C
:10007000C7020008C7020008C7020008C70200083C
:10008000C7020008C7020008C7020008C70200082C
:10009000C7020008C7020008C7020008C70200081C
:1000A000C7020008C7020008C7020008C70200080C
:1000B000C7020008C7020008C7020008C7020008FC
:1000C000C7020008C7020008C7020008C7020008EC
:1000D000C70200089D200008C7020008C7020008E8
:1000E000C7020008C702000800000000C70200089D
:1000F000C7020008C7020008C7020008C7020008BC
:10010000C7020008C7020008C7020008C7020008AB
:10011000C7020008C7020008C7020008C70200089B
:10012000C7020008C7020008C7020008C70200088B
:10013000C7020008C7020008C7020008C70200087B
:1001400000000000000000000000000000000000AF
:10015000C7020008C7020008C7020008C70200085B
:10016000C7020008C7020008C7020008C70200084B
:10017000C7020008C7020008C7020008C70200083B
:10018000C7020008C7020008C7020008C70200082B
:10019000C7020008C7020008C7020008C70200081B
:1001A000C7020008C7020008C7020008C70200080B
:1001B000C7020008C7020008C7020008C7020008FB
:1001C000C7020008C7020008C7020008C7020008EB
:1001D000C7020008C7020008C7020008C7020008DB
:1001E000C7020008C7020008C7020008C7020008CB
:1001F000C7020008C7020008C7020008C7020008BB
:10020000C7020008C7020008C7020008C7020008AA
:10021000C7020008C7020008C7020008C70200089A
:10022000C7020008C7020008C7020008000000005B
:10023000C7020008C702000800000000C70200084B
:10024000C7020008C7020008C7020008C70200086A
:10025000C7020008C7020008C7020008C70200085A
:10026000C7020008C7020008C7020008C70200084A
:10027000C7020008C7020008C7020008000000000B
:10028000C702000800000000C702000800000000CC
:1002900000000000C7020008DFF80CD000F07EF874
:1002A00000480047A9230008700B00240648804737
:1002B00006480047FEE7FEE7FEE7FEE7FEE7FEE74B
:1002C000FEE7FEE7FEE7FEE7CD180008990200080A
:1002D0002DE9F05F0546002092469B46884606467B
:1002E000814640241BE0284641464746224600F00E
:1002F00045F853465A46C01A914110D31146184644
:10030000224600F02CF82D1A67EB01084F462246D2
:100310000120002100F023F817EB00094E41201EB8
:10032000A4F10104DFDC484631462A464346BDE8D5
:10033000F09F30B50B46014600202022012409E041
:1003400021FA02F59D4205D303FA02F5491B04FA8E
:1003500002F52844151EA2F10102F1DC30BD202A6D
:1003600004DB203A00FA02F1002070479140C2F10C
:10037000200320FA03F3194390407047202A04DB3E
:10038000203A21FA02F00021704721FA02F3D0400E
:10039000C2F120029140084319467047064C074DB0
:1003A00006E0E06840F0010394E807009847103445
:1003B000AC42F6D3FFF774FF34250008642500082B
:1003C000FEE70000F0B5BFF34F8FBFF36F8F1D49FD
:1003D00000200860BFF34F8FBFF36F8F1A4C216866
:1003E00041F400312160BFF34F8FBFF36F8F164987
:1003F00070310860BFF34F8F081F006843F6FF7528
:10040000104E1036C0F34E31C0F3C90305EA411255
:10041000184642EA80773760401EFAD2491EF5D26C
:10042000BFF34F8F206840F480302060BFF34F8FC0
:10043000BFF36F8F03484C30016841F00401016045
:10044000F0BD000050EF00E014ED00E07047000048
:1004500010B528B190F83510022903D080214165EC
:10046000012010BD1D4A4FF4956301688C189C4211
:1004700007D8042280F83520086820F001000860C1
:1004800029E00C6824F00E040C6001680A440A6834
:1004900022F001020A60016E0A6822F480720A608A
:1004A00090F85C30012202FA03F10D4B1960D0E99B
:1004B00019134B60C16E31B10B6823F480730B606C
:1004C000D0E91C134B60002180F8341080F83520EF
:1004D000016D01B18847002010BD0000F0FFFDBF95
:1004E000045402580248016841F00101016070475C
:1004F000200400582DE9F84F6C4C00224FF0B04A10
:100500004FF0010B4FF0030E4FF00F090B680BFA81
:1005100002F73B40BB4270D14D68022D01D0122D35
:1005200012D1D50800EB850CDCF820605507ED0EE4
:1005300009FA05F826EA0806D1F8108008FA05F845
:1005400048EA0608CCF82080D0F80080560091F8E0
:1005500004C00EFA06F50CF0030C28EA05080CFAA4
:1005600006FC4CEA080CC0F800C0D1F804C0BCF18D
:10057000010F08D0BCF1020F05D0BCF1110F02D061
:10058000BCF1120F16D1D0F808C0D1F80C802CEABB
:10059000050C08FA06F848EA0C08C0F80880D0F8FC
:1005A00004C02CEA070C0F79C7F30017974047EAFD
:1005B0000C074760C768AF438D68B5403D43C560D1
:1005C0004D68ED006BD53A4D2E6846F002062E6060
:1005D0002D6822F0030606F1B04605F002050095ED
:1005E000D6F808C495072F0F09FA07F52CEA050C71
:1005F000304DA84202D100252EE050E02E4DA842F9
:1006000001D1012528E02D4DA84201D1022523E08A
:100610002B4DA84201D103251EE02A4DA84201D14D
:10062000042519E0284DA84201D1052514E0274DE5
:10063000A84201D106250FE0254DA84201D107258A
:100640000AE0244DA84201D1082505E0224DA84228
:1006500001D1092500E00A25BD4045EA0C05C6F890
:10066000085425684E689D43F60300D51D43256058
:1006700065684E689D43B60300D51D436560DAF892
:10068000005056464F689D43FF0200D51D4335601C
:1006900075684F689D43BF0200D51D437560521CAD
:1006A000102AFFF433AFBDE8F88F00008000005837
:1006B000F44402580000025800040258000802588E
:1006C000000C02580010025800140258001802587A
:1006D000001C0258002002580024025800690840FB
:1006E00000D00120704742694A40426170470AB118
:1006F000018370474183704701488068704700005C
:100700001400002402488168027811448160704717
:1007100014000024032010B500F0A2F80F2000F010
:1007200007F808B1012010BD00F06CF8002010BDE2
:1007300070B50D4D04464FF47A712878B1FBF0F096
:100740000A490968B1FBF0F000F0D0FD48B9102C5F
:1007500007D200222146501E00F062F800206C6093
:1007600070BD012070BD00001400002400000024B2
:10077000134A41781160111D03780A1DE3B14368E3
:100780000B60017BC37A090741EA0361837A41EA7E
:10079000C341437B41EA8341837B41EA4341C37BBD
:1007A00041EA0341437A41EA0321037A007841EAAE
:1007B00043010143116070470020086010607047DA
:1007C00098ED00E0BFF35F8F0448016821F48031A9
:1007D00001600249002070310860704724ED00E09C
:1007E000074940F00100086005487038016841F48D
:1007F00080310160BFF34F8FBFF36F8F70470000F0
:1008000094ED00E07047002809DB012100F01F0291
:1008100091404009800000F1E020C0F800117047CD
:100820000E4BF0B41B68C3F30223C3F10704042C7E
:1008300000D904241D1D072D01D2002300E0DB1E7A
:10084000012606FA04F56D1E0D409D409E40761E61
:10085000164045EA0601F0BC01F068BC0CED00E072
:10086000064A00F0070110684FF6FF03184040EAFF
:100870000120034908431060704700000CED00E0C0
:100880000000FA0510B500F05BFA084909684FF45A
:10089000807292FAA2F201F47061B2FA82F2D1404F
:1008A000034A515CC8400349086010BD184402580F
:1008B0000C2500080000002410B500F0FBF90749E2
:1008C0000968102292FAA2F201F07001B2FA82F2E3
:1008D000D140034A515CC84010BD0000204402587A
:1008E0000C250008364930B50A68096812F0030281
:1008F000344BC1F305311B68334C03F010032468FB
:10090000DFED320AB7EE001AC4F3CC0414FB03F394
:1009100000EE103A2E4BB8EE400A07D02D4C012ABB
:1009200001D0022A4AD0B4FBF1F10BE0244C283C60
:1009300022689506284A03D52468C4F3C104E2401E
:10094000B2FBF1F101EE901A1968B8EE612AC1F319
:10095000080101EE901A1968F8EE611A40EE201AAB
:1009600031EE810A22EE000AC1F34621491C00EE55
:10097000901AF8EE600A80EE201AFCEEC10AC0ED73
:10098000000A1968C1F30641491C00EE901AF8EEFE
:10099000600A80EE201AFCEEC10AC0ED010A196857
:1009A000C1F30661491C00EE901AF8EE600A80EE71
:1009B000201ABCEEC10A80ED020A30BD074ABFE72B
:1009C000284402582C4402583C4402580000003984
:1009D0003844025800093D000090D00340787D0162
:1009E000364930B50A68096812F00302344BC1F386
:1009F00005511B68334C03F480732468DFED320A21
:100A0000B7EE001AC4F3CC0414FB03F300EE103A63
:100A10002E4BB8EE400A07D02D4C012A01D0022AF5
:100A20004AD0B4FBF1F10BE0244C283C2268950637
:100A3000284A03D52468C4F3C104E240B2FBF1F1B3
:100A400001EE901A1968B8EE612AC1F3080101EEAF
:100A5000901A1968F8EE611A40EE201A31EE810AF8
:100A600022EE000AC1F34621491C00EE901AF8EE6E
:100A7000600A80EE201AFCEEC10AC0ED000A196877
:100A8000C1F30641491C00EE901AF8EE600A80EEB0
:100A9000201AFCEEC10AC0ED010A1968C1F3066113
:100AA000491C00EE901AF8EE600A80EE201ABCEEA7
:100AB000C10A80ED020A30BD074ABFE72844025848
:100AC0002C44025844440258000000394044025863
:100AD00000093D000090D00340787D012DE9F047EA
:100AE000DFF8BC9104460E46D9F8000000F007007C
:100AF000B0420CD2D9F8001021F007013143C9F8F7
:100B00000010D9F8000000F00700B0427ED1207834
:100B1000DFF89081800707D5D8F80010E26821F04F
:100B20000F011143C8F800102078C00762D0D8F830
:100B30000010A26821F470611143C8F800105949EF
:100B40006068183902281CD003281DD009680128C4
:100B50001DD04907002960DA524F083F396821F05B
:100B6000070101433960FFF7C7FD0546606841F2A0
:100B70008831022813D003281ED001288A4627D0A6
:100B800034E009688903E5E709688901E2E7C905F6
:100B9000E0E7FFF7B1FD411B514501D923E08A464B
:100BA0003868C0F3C2000228F3D123E0FFF7A4FDA8
:100BB000411B514501D916E08A463868C0F3C2008E
:100BC0000328F3D116E0FFF797FD411B51450AD8E2
:100BD0003868C0F3C2000128F5D10BE0FFF78CFDA7
:100BE000411B514502D90320BDE8F087386810F059
:100BF000380FF3D1D9F80010484601F00701B1428F
:100C00000DD9016821F00701314300E005E00160E2
:100C1000006800F00700B04201D00120E4E720782E
:100C2000400707D5D8F80010226921F07001114360
:100C3000C8F80010207801071B4805D501686269D3
:100C400021F07001114301602178C90605D50168C2
:100C5000A26921F4E061114301602078800607D584
:100C60001149091D0868E26920F07000104308600E
:100C700000F066F8D8F800104FF4807292FAA2F2F1
:100C800001F47061B2FA82F2D140084A515CC84066
:100C9000074908600F20FFF74BFD0020A4E7000084
:100CA00000200052184402581C4402580C25000829
:100CB0000000002410B5FFF7E5FD0849096801228E
:100CC00092FAA2F201F00F01B2FA82F2D140044A84
:100CD000515CC8400349086010BD00001844025828
:100CE0000C2500080400002410B5FFF7E3FF0749B6
:100CF0000968102292FAA2F201F07001B2FA82F2AF
:100D0000D140034A515CC84010BD00001C44025849
:100D10000C25000810B5FFF7CDFF074909684FF40F
:100D2000807292FAA2F201F4E061B2FA82F2D1404A
:100D3000024A515CC84010BD1C4402580C250008F2
:100D40003548F0B50068364D10F03801334809D009
:100D50000411082904D0334E10290BD018290BD0C8
:100D60002046F0BD29688906FBD52968C1F3C10179
:100D7000C840F0BD3046F0BD274918310A680968FF
:100D800012F00302284BC1F305111B68274F03F033
:100D900001033F68DFED260AB7EE001AC7F3CC0760
:100DA00017FB03F300EE103A224BB8EE400A06D0D0
:100DB000012A01D0022A2BD0B4FBF1F008E02A6806
:100DC000920603D52A68C2F3C102D040B0FBF1F00D
:100DD00001EE900A1868B8EE612AC0F3080001EE2F
:100DE000900A1868F8EE611A40EE201A31EE810A76
:100DF00022EE000AC0F34620401C00EE900AF8EEF6
:100E0000600A80EE201ABCEEC10A10EE100AF0BD96
:100E1000B6FBF1F0DCE70000104402580090D0036C
:100E20000044025840787D012C4402583444025852
:100E300000000039304402582DE9F05F0446007884
:100E4000DFF8FC8341F28839DFF8F8A3FE4DC007D4
:100E50004ED0D8F800104046C1F3C20102291AD082
:100E60000068C0F3C200032805D1DAF8000000F0E2
:100E7000030002280FD06068B0F5803F12D010B197
:100E8000B0F5A02F19D0286820F480302860286899
:100E900020F4802009E02868800329D560680028B4
:100EA00074D025E0286840F480302860606890B1F4
:100EB000FFF722FC06464F4609E0286840F48020F0
:100EC0002860EFE7FFF718FC801BB8427DD8286840
:100ED0008003F7D50CE0FFF70FFC06464F4604E011
:100EE000FFF70AFC801BB842F0D828688003F7D4CB
:100EF0002078D64F80075AD5D8F8001040464FF4D6
:100F00007C3B11F0380F13D00068C0F3C2000328F7
:100F100003D1DAF8000080070AD0E068A8B3296896
:100F200021F0190101432960FFF7E6FB06461DE0A9
:100F30002868400702D5E0680028B1D02868E16839
:100F400020F0190008432860FFF7D6FB064604E0AE
:100F5000FFF7D2FB801B0228B8D828684007F7D5D6
:100F600007E0FFF7C9FB801B0228AFD828684007BD
:100F7000F7D538689BFAABF220F47C312069B2FADD
:100F800082F290400143396011E000E0AEE0286851
:100F900020F001002860FFF7AFFB064604E0FFF7F2
:100FA000ABFB801B022891D828684007F7D4207833
:100FB000C00655D5D8F8001040464FF0F84BC1F3A5
:100FC000C201012917D0006800E0EDE0C0F3C200C3
:100FD000032805D1DAF8000000F0030001280AD048
:100FE000E069002828682CD040F080002860FFF7D6
:100FF00083FB064616E02868C00502D5E069802814
:1010000074D138689BFAABF220F0F841206AB2FA4A
:1010100082F290400143396022E0FFF76DFB801BB4
:10102000022899D82868C005F7D538689BFAABF232
:10103000216AB2FA82F220F0F84091400843386009
:101040000EE020F080002860FFF756FB064604E023
:10105000FFF752FB801B022887D82868C005F7D409
:101060002078000724D5774F60694C37002838680E
:101070000FD040F001003860FFF73EFB064604E069
:10108000FFF73AFB801B02288DD838688007F7D518
:101090000EE020F001003860FFF72EFB064604E06A
:1010A000FFF72AFB801B02287ED838688007F7D418
:1010B0002078800623D5A069002828680FD040F446
:1010C00080502860FFF718FB064604E0FFF714FB8A
:1010D000801B022868D828688004F7D50FE020F428
:1010E00080502860FFF708FB064605E0D6E0FFF7D2
:1010F00003FB801B022857D828688004F7D4207887
:10110000400744D5524F386840F480703860FFF78C
:10111000F3FA064604E0FFF7EFFA801B642843D891
:101120003868C005F7D5474FA068483701280AD06E
:1011300008B1052811D0386820F0010038603868FF
:1011400020F0040002E0386840F001003860A06838
:1011500088B1FFF7D1FA064609E0386840F004008C
:101160003860F0E7FFF7C8FA811B49451CD838689A
:101170008007F7D50BE0FFF7BFFA064604E0FFF75C
:10118000BBFA811B49450FD838688007F7D4606ADD
:10119000F0B3D8F80010C1F3C20103297ED00228B1
:1011A000286820F0807000E079E0286003D0FFF725
:1011B000A3FA044687E0FFF79FFA064604E0FFF72C
:1011C0009BFA801B02287BD828688001F7D4DAF8C4
:1011D000001040F2F3329143E26A41EA0211A26A3E
:1011E0001143CAF8001094F834004FF4FE02218E27
:1011F0004002491EA0F5007080B2C1F30801084307
:10120000218F491E02EA0141084394F83C1000E096
:101210005CE0491E120202EA0161084309490831F3
:1012200008600B1D19684FF6F872A06C914392FA92
:10123000A2F2B2FA82F2904001431960014809E03B
:1012400010440258284402580044025804440258EA
:1012500000480258001D0168226C21F00C01114366
:1012600001600168626C21F00201114301600168B4
:1012700041F480310160016841F40031016001688E
:1012800041F480210160016841F00101016028689A
:1012900040F080702860FFF72FFA01E018E00FE0BF
:1012A000044604E0FFF728FA001B022808D8286843
:1012B0008001F7D50AE0FFF71FFA001B022802D9C8
:1012C0000320BDE8F09F28688001F4D40020F8E7EF
:1012D0000120F6E74FF0E0210428086903D020F050
:1012E00004000861704740F00400FAE7401EB0F1C6
:1012F000807F10B501D3012010BD4FF0E024606164
:101300000F21601700F012FF0020A061072020616C
:10131000002010BD7047704790F8791090F87A005F
:101320000843704770B502680446D0691368916835
:1013300010F00F0F64D0594D03F490760D403543F3
:1013400076D0C50707D0DD0505D501251562E26F0A
:1013500042F00102E267820708D5CA0706D0256875
:1013600002222A62E26F42F00402E267420708D5D5
:10137000CA0706D0256804222A62E26F42F0020200
:10138000E26702070ED503F0200201F080552A43E0
:1013900052EAC17206D0256808222A62E26F42F042
:1013A0000802E267E26F002A3AD0800608D503F00F
:1013B000200001F08051084302D0204600F072FB6B
:1013C000E06F000703D42068806840062AD52046D5
:1013D00000F05AFB2068816849061ED5816821F01B
:1013E00040018160606FC0B12D490165606FFFF7FA
:1013F0002FF8002814D0606F016DBDE870400847D9
:10140000850615D503F0200501F0805635430FD031
:101410002046BDE8704000F045BB2046FFF77BFF4B
:1014200070BD05E02046FFF776FF0020E067F7E794
:10143000C6024FF020050CD54E020AD5E803106213
:1014400084F8795084F87A502046BDE87040FFF760
:1014500061BF06060AD503F0800601F400010E43C1
:1014600004D02046BDE8704000F0ACBD41060BD56D
:10147000590609D51168204621F04001116084F811
:10148000795000F005F9CBE70002C9D55800C7D55F
:10149000106820F080401060C2E7000001000010DA
:1014A000751A000810B5040003D094F8790010B143
:1014B00007E0012010BD002084F87800204600F0ED
:1014C00027F8242084F879002068016821F00101C0
:1014D0000160204600F022FB0128EBD0606B10B1C8
:1014E000204600F035FA2068416821F490414160BF
:1014F0002068816821F02A0181602068016841F03C
:10150000010101602046BDE8104000F085BA0000EE
:1015100010B5006886B01B49884230D11A4801686E
:1015200041F001010160006800F0010005901648DB
:101530001030016841F01001016000680121134C76
:1015400000F0100005904FF4007000900220CDE9EB
:10155000010103900720694604902046FEF7CAFF68
:101560004FF48061204600916946FEF7C3FF2520B5
:10157000FFF749F9032225201146FFF751F906B07C
:1015800010BD000000100140E04402580000025865
:1015900090F87A30202B4CD1B9B1B2B190F87830B4
:1015A000012B46D0012380F878304166A0F86820EE
:1015B000A0F86A20FF228168B1F5805F07D07F2301
:1015C00051B1B1F1805F0CD010E00120704701698A
:1015D00021B940F2FF1107E0016909BBA0F86C20B6
:1015E00004E00169E1B13F21A0F86C100021C1675E
:1015F000222280F87A2080F8781001688A6842F008
:1016000001028A6001680A6892000CD50A6842F4F7
:1016100080720A600068816841F08051816006E054
:10162000A0F86C30E2E7086840F490700860002091
:10163000704702207047000030B5006811498842A9
:101640000CD1114A5088010408D411464FF0000310
:101650004404097806D50A2901D0538030BD40F4EE
:1016600000400DE00D2909D0084DC0F30D04401CC9
:1016700080B2C72829555080EFD830BD40F4804053
:10168000508030BD001001400C00002424000024D4
:101690007047FEE7144870B586B0016841F0040158
:1016A0000160016801F004010591016841F0100139
:1016B0000160006800260325694600F010000590CF
:1016C00008200124CDE900060848CDE90245FEF7CF
:1016D00011FF20206946CDE900060548CDE9024505
:1016E000FEF708FF06B070BDE04402580010025833
:1016F000000802582DE9F0411C4C01251C4E012820
:101700001C4F12D0207848B108213046FEF7E6FF82
:1017100068B120213846FEF7E1FF40B1082130468C
:10172000FEF7DCFF012817D01DE02570ECE70A204A
:1017300000F008FE0020207008213046FEF7CEFFA2
:1017400028B120213846FEF7C9FF18B10BE001206F
:10175000BDE8F0810220FBE720213846FEF7BEFFFE
:10176000012800D125700020F2E7000020000024AD
:1017700000100258000802580E4810B586B00168E3
:1017800041F001010160006869460B4C00F0010066
:101790000590022000900120019002900320039008
:1017A0002046FEF7A7FE012220460221FEF79FFFFA
:1017B00006B010BDE0440258000002582DE9FF4772
:1017C00007461E460CA814460D4690E80007FEF793
:1017D000F9FF01208DF8000000208DF808508DF8E9
:1017E0000C008DF809008DF80D808DF80A00684610
:1017F0008DF80E908DF8014001978DF80B608DF8F3
:101800000FA0FEF7B5FF0420FEF7EAFF04B00020AA
:10181000BDE8F087704770477047000070B5284CEE
:101820009CB0256825F004052560254C00260C3465
:10183000256845F440452560256805F440451B951D
:101840002568AD04FCD5012400940CAD0396240456
:10185000019402240994CDE90A410796082485E8F9
:101860000D00CDE910466846FFF7E6FA88B93F203B
:1018700013900320CDE9140640200101CDE9164064
:10188000CDE9180150201A90022113A8FFF726F97C
:1018900010B101201CB070BD0A48016841F0800100
:1018A00001600848F430016841F0020101600068FD
:1018B00000F002001B90FEF715FE0020EAE7000092
:1018C0000C48025800440258FEF71CBF1C4801682F
:1018D00041F4700101601B49086840F00100086094
:1018E000184A0020103210600A68174B1A400A602C
:1018F000144A18321060121D1060121D1060114A37
:1019000028321060121D1060121D1060121D106030
:10191000121D1060121D1060121D1060121D10604B
:101920000A6822F480220A600649603108600120BA
:101930000649C1F80801C0060149803908607047AE
:1019400088ED00E0004402587FEDF6EA0080005187
:1019500090F83410C90706D001684A68836B22F4F6
:1019600000321A434A6090F83410890706D501689E
:101970004A68C36B22F480321A434A6090F83410EC
:10198000490706D501684A68036C22F480221A438D
:101990004A6090F83410090706D501684A68436C1C
:1019A00022F400421A434A6090F83410C90606D562
:1019B00001688A68836C22F480521A438A6090F826
:1019C0003410890606D501688A68C36C22F4005277
:1019D0001A438A6090F83410490611D501684A68A4
:1019E000036D22F480121A434A60016DB1F5801F25
:1019F00006D101684A68436D22F4C0021A434A6066
:101A000090F83410090606D501684A68806D22F402
:101A1000002202434A607047F8B500250446C567B6
:101A2000FEF76AFE0746206800686FF07E460007F2
:101A300008D500223B464FF400112046009600F0E6
:101A4000FBFA60B92068006840070AD500223B46CF
:101A50004FF480012046009600F0EEFA08B1032012
:101A6000F8BD202084F8790084F87A00002084F8FA
:101A70007850F8BD10B5806B0021A0F86A10A0F86E
:101A80006210FFF748FC10BD01680A6822F49072EA
:101A90000A6001688A6822F001028A60202180F8C9
:101AA0007A10704710B5B0F86C2090F87A30016861
:101AB000222B05D0088B40F008000883022010BDBF
:101AC000898C8368B3F5805F01D103696BB11140E4
:101AD000426E531C43661170B0F86A10491E090427
:101AE000090CA0F86A1007D015E0436E1140198068
:101AF000416E891C4166EFE701680A6822F4907222
:101B00000A6001688A6822F001028A60202180F858
:101B10007A10FFF791FD002010BD00002DE9F04F75
:101B2000044600688025FD4B0021D4F810C087B022
:101B3000A6680F46D4F81C8046EA0C06D4F814C0F8
:101B4000A26A4CEA080C46EA0C0632430668DFF843
:101B5000D0C306EA0C061643066020684268E668B1
:101B600022F44052324342602268A0699A4201D076
:101B7000266A3043A66AB6F1005F04D1D4E90B6C43
:101B800046EA0C0630439668DFF898C306EA0C066E
:101B9000064396602068C26A666A22F00F023243EA
:101BA000C262E14E2068E14AB04210D1126802F0F0
:101BB0003802182A74D005DCCAB3082A7AD0102A51
:101BC00047D179E0202A7BD0282A7CD17AE0D84EF0
:101BD000B04209D1126802F00702062A73D2DFE888
:101BE00002F053696B6D6F71D24EB04209D1126829
:101BF00002F00702062A66D2DFE802F0465C5E6069
:101C00006264CD4EB04209D1126802F00702062A82
:101C100059D2DFE802F0394F51535557C74EB04201
:101C20000BD1126802F00702062A4CD200E00EE047
:101C3000DFE802F02A4042444648C14EB04209D192
:101C4000126802F03802182A38D0BBDCB4E74FF033
:101C5000010538E0BB4EB04209D1126802F007021C
:101C6000062A30D2DFE802F01026282A2C2EB64EA3
:101C7000B0420BD1126802F00702062A23D2DFE835
:101C800002F003191B1D1F2100251CE098421AD1E8
:101C9000A64A121D126802F00702062A13D202E0B9
:101CA0000CE007E00CE0DFE802F0030507090B0D8C
:101CB000022508E0042506E0402504E0082502E0AE
:101CC000102500E02025DFF864B2A04E9842DFF82E
:101CD00080A2ABF1540B73D1102D31D006DC022D54
:101CE00009D0042D0AD0082D2FD111E0202D29D0A4
:101CF000402D2AD107E0FEF7DFFD13E06846FEF72E
:101D0000F1FD01980EE003A8FEF76AFE049809E0D1
:101D1000DBF800105846890610D50068C0F3C101F1
:101D20002AFA01F0002811D06168894601EB4101CF
:101D300081420AD8B0EB093F07D808E05046F3E7E4
:101D40008448F1E74FF40040EEE7012733E1102D1E
:101D50004FF000084ED006DC022D0FD0042D15D018
:101D6000082D04D12DE0202D4AD0402D13D001277D
:101D7000794AA0F54071914270D9E6E7FEF79CFDE3
:101D8000626A0023414636F812200DE06846FEF7ED
:101D9000A9FD019803E003A8FEF722FE04980023A2
:101DA000616A36F811201946FEF792FA6268090254
:101DB000030241EA10615008181841EB080115E0D0
:101DC00032E0DBF800105846890609D50068002388
:101DD000C0F3C1012AFA01F0616A36F8112015E05A
:101DE000606A002336F8102050460FE00023FEF70B
:101DF0006FFABDE7606A002336F81020554805E009
:101E0000606A002336F810204FF400400021FEF7EE
:101E10005FFA0902020241EA10614FEA5900101804
:101E20004A4641EB0801E1E7E3694FF4004293427F
:101E30004DD1082D23D005DC8DB1012D12D0042DFC
:101E400006D112E0102D35D0202D3AD0402D11D0E2
:101E5000012721F00F00C1F3420108435AE0FEF7C9
:101E600043FF16E0FEF756FF13E06846FEF73AFD23
:101E700001980EE003A8FEF7B3FD049809E0DBF833
:101E800000105846890608D50068C0F3C1012AFA37
:101E900001F0616A36F8111010E0606A36F810102F
:101EA000BAFBF1F04100606801EB5001B1FBF0F0CA
:101EB00081B2CEE7606A36F810102648B0FBF1F028
:101EC000F0E7606A36F81000B2FBF0F0EAE7082DA0
:101ED0004AD00ADC0DB3012D43D0042D7FF44DAF61
:101EE0006846FEF7FFFC019809E0102D52D0202D26
:101EF00055D0402DF2D103A8FEF772FD0498616A17
:101F000036F81110B0FBF1F1606801EB5001B1FB44
:101F1000F0F080B22168C8604DE01FE0000C00586E
:101F2000F369FFCFFFF4FF11001001405444025841
:101F30000044004000480040004C00400050004079
:101F40000014014000780040007C00401C2500087F
:101F50000090D00300093D00FFFC0F00FEF7C4FE17
:101F6000CDE7FEF7D7FECAE7DBF800205946920618
:101F70000AD50968C1F3C1022AFA02F1626A36F889
:101F80001220B1FBF2F20FE0616A36F81120BAFBC1
:101F9000F2F209E0616A36F811200949F1E7616A55
:101FA00036F81110B2FBF1F2616802EB5102B2FB9C
:101FB000F1F189B2C16007B03846BDE8F08F00008A
:101FC00000093D0090F87910212901D002207047C6
:101FD000B0F8621021B18168B1F5805F13D014E0D0
:101FE00001680A68920004D58A6822F400028A60B7
:101FF00003E00A6822F080020A600068016841F08C
:10200000400101600CE0016961B1C16D4A1CC2650B
:10201000026809781185B0F86210491EA0F86210B4
:1020200000207047C16D02680988C1F3080111855D
:10203000C16D891CC165EEE72DE9F0411E461746CA
:1020400088460446069D1CE0681C1AD025B1FEF7A0
:1020500053FB801BA84214D92068016821F4D07179
:1020600001602068816821F001018160202084F8EE
:10207000790084F87A00002084F878000320BDE815
:10208000F0812068C16938EA010004D00020B8421C
:10209000DAD00020F3E70120F9E7000070B50D4D1C
:1020A00000240D48FFF73EF902E0641CAC4204D85E
:1020B0000948FFF731F92028F7D1002402E0641C19
:1020C000AC4206D8054901220348FFF761FA00280F
:1020D000F5D170BDFFFF0100EC0000240C000024CE
:1020E000FEE700000FB4054B10B503A9044A02989F
:1020F00000F03CF810BC5DF814FB000095230008CC
:10210000100000240FB4084B10B504A902AA0398CC
:1021100000F02CF8044602A9002000F003F9204644
:1021200010BC5DF814FB0000252300080907090E08
:10213000002804DB00F1E02080F80014704700F074
:102140000F0000F1E02080F8141D704702E008C87D
:10215000121F08C1002AFAD170477047002001E021
:1021600001C1121F002AFBD1704700002DE9FF4F6B
:102170008BB09A460F460546002606E025280BD070
:1021800052460D9990476D1C761C28780028F5D191
:102190000FB03046BDE8F08F0024A0460122604910
:1021A00000E0044315F8013F203B02FA03F0084227
:1021B000F7D128782E2817D115F8010F44F0040420
:1021C0002A280ED06FF02F022878A0F130010929BB
:1021D0000AD808EB880102EB410100EB01086D1CF5
:1021E000F2E757F8048B6D1C287869283ED006DC8E
:1021F0000028CDD063280BD0642804D136E07328A2
:1022000010D075284BD052460D999047761C85E02A
:1022100017F8040B8DF8000000208DF80100E94646
:10222000012003E057F8049B4FF0FF3061074FF0A7
:10223000000401D40AE0641C44450DDA8442FADB50
:1022400019F804100029F6D106E0641C8442FCDB76
:1022500019F804100029F8D1264404E019F8010BFC
:1022600052460D999047641EF8D257E001CF4FF0C7
:102270000A0B002802DA40422D2102E0210504D594
:102280002B218DF82410012103E0E10705D0202146
:10229000F7E70DF1200908910CE00021F9E701CFE3
:1022A0004FF00A0BF9E75946FEF743F801F1300207
:1022B00009F8012D0028F6D1ADEB090000F1200B43
:1022C000600701D44FF00108D84502DDA8EB0B00F0
:1022D00000E000208046002406E009A85246005D88
:1022E0000D999047641C761C08988442F5DB04E045
:1022F000302052460D999047761CB8F10001A8F1A4
:102300000108F5DC05E019F8010B52460D999047DC
:10231000761CBBF10001ABF1010BF4DC6D1C34E762
:10232000092801000A68531C0B60107070470000F8
:1023300010B504460420FEF7CDFF0148046010BD2F
:102340000800002470B5002405464FF47A7603E0B7
:10235000304600F005F8641CAC42F9D370BD0000B3
:1023600070B54FF0E02500216C69094AAB6912682D
:102370005043AA699A42FCD002D2A3EB020302E0C6
:10238000A4EB02063344194413468142F1D370BDD5
:10239000080000240349CA695206FCD5C2B20A8566
:1023A00070470000001001400EB50024FEF70AF847
:1023B000FEF7B0F9042302220521A020FFF72EFA30
:1023C0004FF4C870FFF7B4FF4FF4E13000F082F82B
:1023D000FFF7D2F9FFF75EF91EA0FFF783FEDFF8E3
:1023E0008890002501264FF0202832270020FFF793
:1023F00081F9012811D002281CD00A20FFF7A2FF82
:10240000641CE4B2B4FBF7F007FB10400028EDD1E8
:1024100002214846FEF767F9E8E700950623012206
:1024200040468021CDE90156FFF7C8F90FA0FFF71C
:1024300059FEE5E710A0FFF755FE1A4814A1224601
:10244000FFF760FE18A0FFF74DFE16491CA0FFF72E
:1024500049FED5E70D0A0D0A4D505520636C6F7388
:102460006564210D0A000000000002584D505520FF
:102470006F70656E210D0A0053746172742057727B
:102480006974696E6720646174612E2E2E0D0A00D6
:102490004D505520746573742061727261792025E6
:1024A00064000000002000204461746120577269BC
:1024B00074652066696E73686564210D0A0000000A
:1024C000417272617920646174612069733A257385
:1024D0000D0A00000B490A4A10B5C1E9002000208E
:1024E0008860C860086188610C2048610846FEF772
:1024F000D9FFBDE81040044901220248FFF748B85F
:1025000000100140EC0000240C000024000000003A
:102510000102030401020304060708090100020086
:102520000400060008000A000C0010002000400013
:102530008000000164250008000000242400000041
:102540004C210008642500080000002080200000C5
:102550005C21000888250008240000244C0B0000A2
:102560005C2100080090D0030090D0030000000020
:10257000000000000000000001000000100000004A
:08258000000000000100000052
:040000050800029954
:00000001FF
